:100000000AC115C015C015C015C015C015C015C052
:100010002FC02FC02FC0444D42393020496E746527
:1000200072666163652056312E300D0A0000189506
:10003000189518951895189518954F934FB74F9395
:100040004CB14CB94D3029F04A3019F0883260F487
:1000500002C0C09409C0AF93BF93BB27A0E8A80F0C
:100060004C938395BF91AF914F914FBF4F9118958E
:1000700018951895189540534A3010F04F7D475009
:1000800008955F936F935FB75F9352EC65E05A9565
:10009000F1F76A95E1F75F915FBF6F915F91089506
:1000A0005F935FB75F9356E05A95F1F70000000049
:1000B0005F915FBF5F9108955F935FB75F9355E76F
:1000C0005A95F1F7000000005F915FBF5F910895BE
:1000D000C895002021F03196602D02D0F9CF089507
:1000E0006CB9CFDF089548E0660F10F48D9801C019
:1000F0008D9A8C9AE1DF8C98DFDF4A95A9F70895F5
:1001000048E08C9AD9DF0894839B889467958C98F3
:10011000D3DF4A95B1F7089541B3437C41BB49E130
:10012000CBDF4A95E9F741B34C6341BBB9DF41B33B
:100130004B7E41BBB5DFB4DF40B3447006C041B372
:10014000437C41BB6DE2CCDF08956BE2C9DF41B374
:100150004F7D41BBA5DF41B3477F41BBA1DFA0DF9E
:1001600041B34C6041BB40B34071E9F740B34071CB
:10017000E9F349E1A1DF4A95E9F741B3437F41BB88
:100180004FE08EDF4A95E9F76AE5ADDF95DF94DF52
:1001900093DF6BEBA8DF90DF8FDF8EDF6FEFA3DFE6
:1001A00041B34F7C41BB88DF40B34071E9F342E18A
:1001B00083DF4A95E9F7B8E0A4E1A2DF6CB94FE02C
:1001C0006FDF4A95E9F71197C1F741B3437C41BB13
:1001D0000895BB27A0E8882309F41CC07D917F7D8A
:1001E000743409F406C07C3409F403C0763591F404
:1001F00000C0743411F490DF0DC07C3429F440E465
:10020000A2B2A426A2BA31F4763521F43ADFE6E1AF
:10021000F0E05EDF0895F8944FED4DBF789447E12C
:1002200049B948E94AB940E442BB40E441BB4FEF19
:1002300047BB40E048BBCC20F1F3CC2444E621DFAF
:0A0240004A95E9F7C6DF8827F6CFDC
:00000001FF
